:020000001629BF
:1000080009008A018207613400340B344134013419
:100018000B34483402340B34623403340134593419
:1000280004340B3443340534013464340634013465
:10003800653407340934453408340F3466340934D8
:10004800013479340A340B3467340B34013468349E
:100058000C34013469340D340B346A340E340134F1
:100068006B340F3401346C3410340B346D34113468
:100078000B346E3412340B344E3413340B346F3467
:1000880014340B344F3415340B34703416340134B3
:10009800723417340634523417340F347334183426
:1000A800013453341934013474341A340134543457
:1000B8001B34013478342234013475341C34073449
:1000C80055341C34123476341D340B3477341E34D2
:1000D8000A3457341E3414347A341F340B345A34E7
:1000E80020340B344B34213401342034FF340034B1
:1000F8002E34FF3401340034003400348A0182077E
:0601080077297A292E2957
:100200008A010A148200533479346E343134303424
:1002100034343E3400344C346F34613464346934E3
:100220006E3467342E342E342E340034831601306D
:100230008500103087008E308100003090005030F3
:100240009F00003091008312043092002011871625
:10025000071404223730AB002430FA222011572132
:1002600003304222BE22E822A4000D3A03192E29AF
:1002700024082F3A031966292408233A031963290D
:100280002408543A03195C292408573A0319CF2942
:100290002408443A0319E1292408533A03190B2A84
:1002A00057213F30FA22193033232E292E290D30C1
:1002B000FA220A30FA220800E00A60082B226400C1
:1002C000071E5C292E294B2295212E29E8227D210B
:1002D000031D6B292E296008FF3A03197429600851
:1002E0009521E10B6B296629610882206629783007
:1002F000332308001E3033230800A600DF018329C2
:10030000DF0ADF0ADF0A5F080520003A0319080048
:100310002606031D8029DF0A5F080520E000DF0AAA
:100320005F080520E100031108009821B3210800AF
:10033000B2000310B20D0310B20D0630B207B101C6
:10034000A22108008712033011223108112232083D
:1003500011221E22A7001E22A8001E22A9001E2272
:10036000AA008716080087120330112228081122DC
:10037000270811221E222B222B08C821A903290F8E
:10038000AA0AAA0329082A04031DBA298716080005
:10039000AC00000000000000AC0BC9290800572188
:1003A0000B304222572187120230112200301122D5
:1003B000003011221023112264002130FA2220156E
:1003C000DA29A701A8018712033011222808112277
:1003D000270811220030A2007D30A3001E222B220C
:1003E0006400FC21A203220FA30AA3032208230412
:1003F000031DEE2987162E293A30AF0000000000B9
:100400000000AF0BFE290800871201301122413095
:100410001122871608008712053011221E22871626
:100420002E29A600A101A115A60D031C0511031874
:10043000051585148510A10B142A0800A101A1152A
:10044000A6010310A60D8514051826148510A10B0E
:10045000212A26080800A40011308714071034222E
:100460002408342207140800A6000830A100A60DB5
:10047000031C071103180715871000008714A10B30
:10048000372A0800DE005E080021003A0319080040
:10049000FA22DE0A432AA601E822A4003030A40290
:1004A000031C5A2A0A30240203185A2A5D222408FF
:1004B000A6074C2AEE22260808000310A60D2608DF
:1004C000A60DA60DA60708002010A60064306C2219
:1004D0000A306C2220140130A4003030B30024080C
:1004E000A602031C752AB30A702AA607330820182F
:1004F000FA2A303A031D2014303A2018FA22080054
:100500000430A100B101B20199220318912AB20D61
:10051000B10DB20DB10DB20DB10DB20DB10DB207ED
:10052000842AEE2208009922A400A40E992224070E
:100530000800E8229C220800D03E031CA82AF63EB0
:10054000031CAC2AF93E031CA82AFA3E031CAB2A62
:10055000031400300800063E0A3E0310080031086C
:10056000B4223208B4220800A600260EB8222608BB
:100570000F39F63E0318073E3A3EFA2AB40110231B
:10058000DD000A3A0319BF2A5D08083A0319D82A80
:100590003408353E84005D088000FA225D080D3A7B
:1005A0000319E62AB40A34084D3A0319E22ABF2A8D
:1005B000B403B41BBE2A0830FA222030FA220830D5
:1005C000FA22BF2A0830FA22B403BF2AB401080075
:1005D0003408353E84000008B40A0800B40308005B
:1005E0009F3E031CF82AE63E0318203E5B3E0800AF
:1005F000613E0800A400A101A115871100000000C0
:100600000000000000002623A40C031C871103181F
:100610008715A10B022B26238715262326230800E6
:10062000A101A115A401201D6400071E132B28237E
:10063000071E102B26230310071E0314A40C000012
:100640000000A10B1A2B2623240808001830292BA0
:100650000C30AF00AF0B2A2B0800AF0064303323FF
:10066000AF0B2E2B0800AE004123AE0B342B08003D
:10067000AE004123AE0B392B08000130422B0A306B
:10068000422B64306400AD000F30AC00AC0B462B45
:080690000000AD0B442B080033
:02400E006A0046
:00000001FF
